:020000040800F2
:10000000D00800209D0100081F1D00088D18000861
:10001000D51C0008970B0008FB2A00080000000010
:10002000000000000000000000000000EB200008BD
:10003000E112000800000000D51D00081922000888
:10004000B7010008B7010008B7010008B7010008B0
:10005000B7010008B7010008B7010008B7010008A0
:10006000B7010008B7010008B7010008B701000890
:10007000B7010008B7010008B7010008B701000880
:10008000B7010008B7010008B7010008B701000870
:10009000B7010008B7010008B701000839140008CB
:1000A000B7010008B7010008B7010008B701000850
:1000B000B70100082D230008B7010008B7010008A8
:1000C000B7010008B7010008B7010008B701000830
:1000D000B70100086D280008B7010008952800083E
:1000E000B7010008B7010008B7010008B701000810
:1000F000B7010008B7010008B7010008B701000800
:10010000B7010008B7010008B7010008B7010008EF
:10011000B7010008B7010008B7010008B7010008DF
:10012000B7010008B7010008B7010008B7010008CF
:10013000B7010008B7010008B7010008B7010008BF
:10014000B7010008B7010008B7010008B7010008AF
:10015000B7010008B7010008B7010008B70100089F
:10016000B7010008B7010008B7010008B70100088F
:10017000B7010008B7010008B7010008B70100087F
:10018000B7010008B7010008DFF80CD000F074FADE
:100190000048004735330008D00800200648804753
:1001A00006480047FEE7FEE7FEE7FEE7FEE7FEE75C
:1001B000FEE7FEE7FEE7FEE761220008890100088E
:1001C0002DE9FE4F804681EA0300C00F0C460090E7
:1001D00021F0004123F00045B8EB0200A94105D20F
:1001E0004046214690461C460B46024623F00040FE
:1001F000104347D0270DC7F30A00C3F30A510290FA
:10020000401A019040286BDAC3F3130040F4801BBE
:100210000098924620B10023D2EB030A63EB0B0B4C
:1002200001985946C0F14002504600F01FF90646B9
:100230000D4650465946019A00F027F910EB080088
:100240006141002487EA115284EAE7731A4340D0DF
:10025000009A62B3019A012A4FEA075215DC001B8B
:1002600061EB02014FF0004202EA0752CDE9004281
:10027000001C41F5801132462B4600F05EF903B0B8
:10028000BDE8F08F40462146F9E7001B61EB020113
:10029000001C41F5801300185B412018A2F50017DF
:1002A00047EB030140EAD570B6196D4111E06D08C6
:1002B0004FEA360645EAC0754FEA0752001B61EB6C
:1002C0000201001C41F5801149084FEA3000001975
:1002D000514132462B4603B0BDE8F04F00F01EB945
:1002E0000098012240000023D0EB020263EBE07390
:1002F000009821464FEAE074B8EB000061EB04017E
:10030000E9E783F000435BE781F0004158E72DE91E
:10031000F04D81EA030404F0004B21F0004514463F
:100320004FF0000A23F0004150EA050220D054EAC1
:1003300001021DD0C5F30A570246C5F31303C1F3EA
:100340001300C1F30A5640F4801543F48013A7EB61
:100350000608101BD64608F2FD3873EB050002D3E1
:1003600008F1010801E092185B41B8F1000F03DACF
:1003700000200146BDE8F08D00204FF480110646B4
:1003800084460EE0171B73EB050705D3121B63EBC6
:10039000050306434CEA010C49084FEA3000921865
:1003A0005B4150EA0107EDD152EA030012D082EA24
:1003B000040083EA0501084305D0101BAB4106D2B7
:1003C0000122002306E000224FF0004302E06FF01C
:1003D000010253101AEB06004CEB085110EB0A0017
:1003E00041EB0B01BDE8F04D00F098B80EB5C10F20
:1003F00080EAE0700844CA07002140F233438DE8E8
:100400000E000A460B4600F098F803B000BD00F05D
:10041000004230F000400AD0C10D01F56071C0F318
:10042000160042EA0151C2084007114370470020FC
:100430000146704701F0004330B421F0004150EA1A
:10044000010206D00A0DA2F56072C1F31301002A61
:1004500002DC30BC00207047440F44EAC104C100F4
:10046000E01830BC00EBC25000F021B8202A04DBB9
:10047000203A00FA02F1002070479140C2F12003B7
:1004800020FA03F3194390407047202A06DBCB176C
:10049000203A41FA02F043EAE07306E041FA02F33F
:1004A000D040C2F12002914008431946704700290C
:1004B000A8BF7047401C490008BF20F001007047EA
:1004C00010B4B0FA80FC00FA0CF050EA010404BF4A
:1004D00010BC704749B1CCF1200421FA04F411FAA0
:1004E0000CF118BF012121430843A3EB0C01CB1DE4
:1004F0004FEA00614FEA102042BF002010BC704755
:1005000000EBC35010440029A4BF10BC7047401C2E
:10051000490008BF20F0010010BC704710B5141E40
:1005200073F1000408DA401C41F1000192185B41AC
:100530001A4301D120F0010010BD2DE9F04D924683
:100540009B4611B1B1FA81F202E0B0FA80F220329A
:100550009046FFF78BFF04460F4640EA0A0041EA47
:100560000B0153465A46084313D0114653EA010083
:1005700019D0C8F14002504600F090F805460E46EA
:10058000504659464246FFF771FF084305D0012007
:1005900004E020463946BDE8F08D0020054346EAD8
:1005A000E0762C4337430A986305E40AA0EB080081
:1005B0000022FD0A44EA47540A3002D500200146D1
:1005C000E9E7010510196941DDE9084500196941AC
:1005D000BDE8F04DA2E72DE9F04D00231A461B1AA5
:1005E0008A4103DB00200146BDE8F08DC1F30A52C9
:1005F000C1F3130141F480154FF0000BD10702D174
:1006000000186D41521E0027044640F2FF11384683
:1006100001EB620A3E468046024600204FF48011FC
:1006200000F03CF8C2197141BB1846EB0100B4EB75
:10063000030C75EB000C04D3E41A65EB00051746B8
:100640000E46241908F101006D4180463428E3DD8F
:10065000F91946EB0600091BA84103D24FF0FF32FF
:10066000134601E0002213461BEB070046EB0A513C
:10067000BDE8F04DFFF752BF064C074D06E0E068BD
:1006800040F0010394E8070098471034AC42F6D3D9
:10069000FFF77EFD903E0008B03E0008202A04DBF4
:1006A000203A21FA02F00021704721FA02F3D040EB
:1006B000C2F12002914008431946704730B58C18AA
:1006C00010F8012B12F00F0301D110F8013B1209B1
:1006D00006D110F8012B03E010F8015B01F8015B73
:1006E0005B1EF9D101E001F8013B521EFBD1A14292
:1006F000E6D3002030BD10B500F058F900F026F820
:1007000000F012F910BD21B1826842F0010282604E
:1007100003E0826822F00102826070470021084AEB
:100720001168084A1140D0E900231A4383681A432C
:10073000C3681A431143044AC2F804137047000007
:1007400004230140E030FCFF0020014000B58BB0E5
:100750000121080201F060FB0121480201F05CFB6D
:100760000121880201F058FB00F014F916200190D5
:100770004FF480300290801003900020049001A874
:10078000FFF7CCFF05A800F0FCF900200590012040
:100790008DF8180000208DF81900099018208DF8A8
:1007A000280000200790089008208DF8280005A94F
:1007B000544800F045F9052301220021514800F07A
:1007C0007FF90523022201214E4800F079F9052323
:1007D000032202214B4800F073F905230422032170
:1007E000484800F06DF905231A460A21454800F0F3
:1007F00067F9052306220B21424800F061F9052321
:1008000007220C213F4800F05BF9052308220D2147
:100810003C4800F055F901213A4800F079F80620EB
:100820008DF8280005A9384800F00AF905230122AF
:100830000621354800F044F90523022207213248F9
:1008400000F03EF90523032208212F4800F038F973
:100850000523042209212C4800F032F905231A4609
:100860000E21294800F02CF9052306220F212648E5
:1008700000F026F908208DF8280005A9234800F08B
:10088000DFF8052301220421204800F019F905238F
:10089000022219461D4800F013F905230322062100
:1008A0001A4800F00DF9052304220721174800F02B
:1008B00007F905231A460821144800F001F9052319
:1008C00006220921114800F0FBF8052307220E211A
:1008D0000E4800F0F5F8052308220F210B4800F020
:1008E000EFF8012000F0D6F801210648FFF70BFFD2
:1008F00001210548FFF707FF01210448FFF703FF27
:100900000BB000BD00200140002101400022014049
:1009100021B1826842F48072826003E0826822F42E
:10092000807282607047000000B58FB00121880599
:1009300001F052FA002000900390182004904FF428
:100940008070099040020A900F48019000200590A5
:100950004FF40060079000200E900C4802904FF476
:1009600080600690C000089000200D900B90012040
:100970000C906946064800F0D1FA0121044800F0C5
:1009800007FA0FB000BD00000823014084020020D8
:100990001064024010B50121080201F04DFA002157
:1009A0004FF4807001F048FA10BD00001CB5012121
:1009B000084601F011FACF20009003208DF80400C2
:1009C00000208DF807006946194800F0E9FD012173
:1009D000022001F001FA032000908DF804000020AD
:1009E0008DF807006946134800F0DAFD0121042064
:1009F00001F0F2F93F20009003208DF80400002060
:100A00008DF8070069460C4800F0CAFD012120203E
:100A100001F0E2F94FF4FF60009003208DF804002C
:100A200000208DF807006946044800F0B9FD1CBDA0
:100A3000000002400004024000080240001402408E
:100A400030B50246002000235068104C20400D793C
:100A50000C6844EA05242043506090680C4C204008
:100A6000D1E903542C438D682C434D7944EA450465
:100A700020439060D06A20F470000C7D641EE4B2C4
:100A8000234340EA0350D06230BD0000FFFEFFFC6C
:100A9000FDF7FFC038B10849096841F40051074A21
:100AA000C2F8041306E00449096821F40051034A1E
:100AB000C2F80413704700000423014000200140E5
:100AC000F0B504460D4600200021092D11DDE06837
:100AD000A5F10A0606EB4607072606FA07F1884342
:100AE000A5F10A0606EB460603FA06F10843E060A4
:100AF0000CE0206905EB4507072606FA07F1884355
:100B000005EB450603FA06F108432061072A0FDAD0
:100B1000606B561E06EB86071F2606FA07F1884310
:100B2000561E06EB860605FA06F10843606322E0CE
:100B30000D2A0FDA206BD61F06EB86071F2606FA52
:100B400007F18843D61F06EB860605FA06F108432F
:100B5000206310E0E06AA2F10D0606EB86071F266F
:100B600006FA07F18843A2F10D0606EB860605FAA0
:100B700006F10843E062F0BD816841F08041816088
:100B8000704700210160017141718160C1600161A4
:100B900001210175704700BFFEE7000000B5034664
:100BA00008480088984206D04FF6FF70834202D072
:100BB0000BB1B12B01D1012000BD00F069FE002076
:100BC000FAE70000660000200120704710B52DED07
:100BD000028BB0EE408AF0EE080A88EE200ADFEDC4
:100BE0000A0A20EE200ABCEEC00A10EE100A84B2F7
:100BF0002146002000F07CF80121002000F098F848
:100C0000BDEC028B10BD000000F07F4539B1084AF1
:100C10001268012383401A43054B1A6006E0044A18
:100C20001268012383409A43014B1A607047000009
:100C30000074004000B587B00121084601F0CCF8EF
:100C40000121480701F0D8F83020059003208DF8E5
:100C5000180000208DF81B0003208DF819000020DB
:100C60008DF81A0005A9144800F09AFC3C20019068
:100C700000200290049001A900F020F801A91020A2
:100C800000F01CF801210020FFF7C0FF0121102017
:100C9000FFF7BCFF0021084600F02AF800210846B3
:100CA00000F036F80121002000F042F80121102068
:100CB00000F03EF807B000BD0000024030B5002251
:100CC00000230A4C226840F6FE748440A243D1E916
:100CD00000452C438D682C43CD6844EA050303FA94
:100CE00000F42243014C226030BD0000007400403B
:100CF00008B500220092054A009200F10802009B0C
:100D00001A440092009A116008BD0000007400406F
:100D100008B500220092054A009200F11402009BDF
:100D20001A440092009A116008BD0000007400404F
:100D300010B541B1084A126804090123A3401A43BF
:100D4000054B1A6007E0044A126804090123A34016
:100D50009A43014B1A6010BD047400400246094BCF
:100D60009A4201D2084801E00648103801F00053C9
:100D70001BB1064B0B40C36002E0044B0B40836089
:100D80007047000010640240006002407D0F7D0F3C
:100D900021B1026842F00102026003E0026822F021
:100DA0000102026070470000016821F0010101604A
:100DB0000021016041608160C160016121214161C8
:100DC0004A49884204D13D21484A103A91608CE05A
:100DD00046491831884205D14FF47461434A103AAC
:100DE000916082E041493031884205D14FF474115D
:100DF0003E4A103A916078E03C494831884205D13A
:100E00004FF07461394A103A91606EE037496031B1
:100E1000884204D13649354A103AD16065E03349F9
:100E20007831884204D13349304A103AD1605CE0CD
:100E30002E499031884204D12F492C4A103AD16072
:100E400053E02A49A831884205D14FF03D51274A45
:100E5000103AD16049E02949884204D13D21274A0E
:100E6000083A116041E025491831884205D14FF414
:100E70007461224A083A116037E0204930318842D3
:100E800005D14FF474111D4A083A11602DE01B4939
:100E90004831884205D14FF07461184A083A116010
:100EA00023E016496031884204D11149134A121FC8
:100EB00011601AE011497831884204D10D490F4A76
:100EC000121F116011E00D499031884204D10A4986
:100ED0000A4A121F116008E00849A831884204D16B
:100EE0004FF03D51054A121F1160704710600240DB
:100EF0003D000020400F002000003D201064024013
:100F0000014600200A6802F001020AB1012000E057
:100F1000002070470146486880B2704710B5002233
:100F20000268134B1A40CC680B6823434C69234377
:100F30008C692343CC6923430C6A23434C6A2343C3
:100F40008C6A23434C6B23438C6B23431A4302600C
:100F5000426922F00702D1E90B3423431A4342616C
:100F60000B6943604B6883608B68C36010BD0000F1
:100F70003F801CF04160704710B500210F48FFF71B
:100F800007FF01200E4908700C48FFF7C3FFC0F1AE
:100F90000A000C49087000200B490A4A127888544C
:100FA0000A210648FFF7E6FF4FF081510348FFF79B
:100FB000D5FE01210148FFF7EBFE10BD286002407D
:100FC00057000020580000209401002010B52D4843
:100FD000007848B902F0CEFB00202B4908600121BF
:100FE0002A4800F051FB4CE026480078012837D110
:100FF000274890ED000ADFED270AB4EEE00AF1EE93
:1010000010FA03D20121214800F040FB1D4800786E
:10101000012805DB2048007810B901201E4908701E
:101020001E48007850B91E48007810B900F0AEFA9A
:1010300001E000F085FF02F0B3FB22E017480078E2
:1010400001280AD11648007810B900F09FFA01E093
:1010500000F076FF02F0A4FB13E002F08BFB10E03F
:1010600008480078022802D102F0E0F809E00548BB
:101070000078032802D102F015F902E000200149AE
:10108000087010BD810000202401002000180240DB
:10109000600100206F12833A2801002083000020A5
:1010A0008400002030B58FB07748007800287DD0CC
:1010B000FFF78AFD01287AD1734800780B2877D290
:1010C000DFE800F0DB066286AFC5D8D9DBDBDA00EB
:1010D0004FF400616D4800F0D9FA02206C490860B5
:1010E0000024002500206B49087000F0DBFA05465B
:1010F00000BF07E004F109006749085C0DF804002F
:10110000601CC4B2AC42F5DB9DF800006349087076
:101110009DF80100624908709DF80200614908705D
:101120009DF80300604908600846006800020860F6
:101130009DF80400096808445B4908609DF80500B3
:101140005A49086008460068000208609DF80600D9
:1011500009680844554908609DF80700544908602B
:1011600008460068000208609DF808000968084405
:101170004F49086001204F4908604F48006820F03F
:1011800040004D49086079E002204149086042482A
:10119000407A4A490860084690ED000AB8EE400AD5
:1011A000DFED470A80EE201A464802E069E066E07B
:1011B00063E080ED001A01204349087002203D4998
:1011C00008603D48006820F040003B49086055E059
:1011D0004FF400612D4800F059FA02202C490860B4
:1011E0003548006840F04000334908602A48407A9A
:1011F000364908702848807A64280BDC2648807AB3
:1012000000EB80000001642190FBF1F06E3030496A
:10121000086002E0BE202E490860032025490860CE
:101220002CE04FF40061194800F030FA0020184912
:1012300008601948407A2749087001201D49086054
:101240001D48006820F040001B49086016E0124865
:10125000407A214908600846006828B94FF4C04127
:101260001E4800F011FA04E04FF4C0411B4800F0A2
:101270000DFA03E002E001E000E000BF00BF00F073
:1012800007FB0FB030BD00006900002000140240D1
:101290002001002062000020480200208100002080
:1012A0008300002084000020880000208C000020A3
:1012B0009000002098000020003C0140A000002089
:1012C0000000C842A4000020680000208200002026
:1012D0009C000020800000205001002000100240EF
:1012E00070470021002200BF05E0002200E0521CF0
:1012F0000A2AFCDB491C8142F7DB704730B5044603
:101300004748006820B1012817D0022872D132E086
:10131000052C11D14348006820F040004149086085
:1013200000204149086041480968445401203C4973
:10133000086000203E4908606EE03B480068401CA1
:101340003949086039480968445437480068022818
:1013500010D302203249086034488178407801EB8C
:10136000002033490860084600683B2802D300F09B
:101370008FFA30BD50E02C480068401C2A490860B4
:10138000084600683B2802D300F082FAF1E72748BC
:101390002549096844542448006825490968884259
:1013A00036D3224845792D02807905432846FFF738
:1013B000F5FB48B300231D48C3791B02007A0344A0
:1013C0006FF470401844052819D2DFE800F00307D5
:1013D0000B0F140001201749087013E00220154973
:1013E00008700FE00320134908700BE00420114936
:1013F000087007E00DE005200E49087002E000F0DB
:1014000047FA00BF00BF02E000F042FAB1E700BFB8
:1014100002E000F03DFA00BF00BF00BFA9E70000F6
:1014200070000020003C01407400002048020020B1
:101430007C0000206900002010B5402000F012F868
:1014400038B104480068401C02490860402000F0A0
:1014500003F810BD14010020014908607047000026
:10146000143C014001460020034A12680A400AB1B8
:10147000012000E000207047143C01400021234976
:101480008279002A3AD00A46126803689A430B46CA
:101490001A600A1D126803689A430B1D1A600279CC
:1014A00011440A6803681A430A60184A083212682D
:1014B00003689A43154B08331A601A1D12680368B3
:1014C0009A43124B0C331A604279102A0ED11A1F1C
:1014D000126803681A430D4B08331A601A1D12680C
:1014E00003681A43094B0C331A600DE0074942792F
:1014F00011440A6803681A430A6005E0027911443E
:101500000A6803689A430A6070470000003C014083
:1015100000B585B04FF4C06000F052FC17208DF884
:10152000100001208DF8110003208DF81200012019
:101530008DF8130004A800F007FC0121042000F03E
:101540004BFC0121880300F067FC40200290002042
:101550008DF80C008DF80F0002A90B4800F020F860
:101560000621022000F0C2FD4020009000208DF8EE
:10157000040008208DF8050001208DF8060068465B
:10158000FFF77CFF05B000BD0008024010B54FF426
:101590000051024800F078F810BD0000000C024035
:1015A000F0B50A4600210023002400BF3DE00125DC
:1015B00005FA01F3156805EA03049C4234D1056875
:1015C0004F000326BE40B543056015794E00B54077
:1015D0000668354305601579012D02D01579022D75
:1015E00016D185684F000326BE40B5438560557906
:1015F0004E00B540866835438560456801268E40BB
:10160000B5434560456896798E40B6B2354345602E
:10161000C5684F000326BE40B543C560D5794E006E
:10162000B540C6683543C560491C1029BFD3F0BD1D
:10163000F0B5002300244D07ED0E02FA05F3CE109D
:1016400000F1200555F826504E07F70E0F26BE4034
:10165000B543CF1000F1200646F82750CE1000F118
:10166000200555F8265045EA0304CE1000F1200568
:1016700045F82640F0BD0246002013690B400BB12F
:10168000012000E0002070474183704701837047CC
:1016900042694A40426170470AB1018300E04183D8
:1016A00070470000002104488278407802EB002057
:1016B0000B3881B2C8B27047480200201CB5012126
:1016C000084600F089FB0121022000F085FB012182
:1016D000042000F081FB0121082000F07DFB0121A6
:1016E000102000F079FB0121202000F075FB012182
:1016F000402000F071FB0121802000F06DFB0320F1
:10170000009002208DF8040001208DF806000020D2
:101710008DF8070002208DF8050069465548FFF74F
:101720003FFF40F60400009001208DF804000020E7
:101730008DF806008DF8070002208DF80500694637
:101740004C48FFF72DFF0420009001208DF8040085
:1017500000208DF806008DF8070002208DF80500A6
:1017600069464548FFF71CFF0320009001208DF8D3
:10177000040000208DF806008DF8070002208DF887
:10178000050069463D48FFF70BFF4FF4C05000903D
:1017900000208DF804008DF8070002208DF8050068
:1017A00069463748FFF7FCFE4FF4C0400090012027
:1017B0008DF8040000208DF8070002208DF8050048
:1017C00069462F48FFF7ECFE4FF4C040009001201F
:1017D0008DF8040000208DF806008DF807008DF8C4
:1017E000050069462748FFF7DBFE4FF48050009064
:1017F00000208DF804008DF8070003208DF8050007
:1018000069462048FFF7CCFE4020009000208DF86C
:10181000040001208DF8070002208DF805006946BC
:101820001948FFF7BDFE04211348FFF72DFF4FF4C1
:10183000C0411448FFF728FF4FF400411048FFF75C
:1018400023FF4FF400610B48FFF720FF03210B48F3
:10185000FFF71AFF4FF480410A48FFF717FF0421F2
:101860000448FFF711FF4FF4C0410548FFF70CFF94
:101870001CBD000000140240000402400018024099
:1018800000100240000C02400008024000BFFEE7CA
:101890000020114908701149086011490860114978
:1018A0000860114908701149087011490860114910
:1018B000086009E0002010490E4A126888540D485B
:1018C0000068401C0B4908600A4800683C28F1D3B6
:1018D000002008490860704769000020740000205B
:1018E000700000207C0000205F00002060000020CD
:1018F0006C000020780000204802002010B5D121A3
:10190000802000F07FF910BD70B52DED108B84B0F4
:1019100000249FED5E0AF0EE40FA9FED5D0AB0EE06
:1019200040FA9FED5C0AF0EE409A012000F006F9C3
:101930000402022000F002F90443640800EE104A99
:10194000F8EE400A9FED541A80EE810ADFED530A4B
:1019500020EE200AF0EE408AB1EE4F0A10EE105A47
:101960002FEE0F0AF1EE000A00EEE90A8DED030AF0
:10197000B1EE000A29EE800AC0EE2F0ACDED020A70
:10198000B0EE000A29EE800A10EE106A9DED030AFF
:10199000DDED020A00EEA80AB0EE409A3046FEF7EE
:1019A00036FD41EC1B0B2846FEF731FD41EC1D0BCB
:1019B00019EE100AFEF72BFD41EC1E0BB0EE4E0A9D
:1019C000F0EE6E0A01F09BF88DED000B53EC1D2B31
:1019D0009DED000B51EC100BFEF7F2FB41EC1C0BE4
:1019E00053EC1B2BFEF793FC41EC1A0BFEF722FD88
:1019F00009EE100AB5EEC09AF1EE10FA05DBB0EE72
:101A0000490A04B0BDEC108B70BDB0EE688A9FED42
:101A1000240AB0EE409ADFED230AB0EE490A00EE48
:101A2000880AB0EE409A28EE280AB0EE408ADFED30
:101A30001E0AB0EE490A00EE880AB0EE409A28EE7F
:101A4000280AB0EE408ADFED190AB0EE490A00EE2E
:101A5000C80AB0EE409A28EE280AB0EE408ADFEDC0
:101A6000140AB0EE490A00EEC80AB0EE409A28EE19
:101A7000280AB0EE408ADFED0F0AB0EE490A00EE08
:101A8000880AB0EE409AB0EE490ABAE70000C842B0
:101A90003211803B7F051BB5000000470000C843A2
:101AA0001F0572C35B420E403478293B06EFA13616
:101AB0001317F2323B99272F1CB501210A2000F0A1
:101AC0008BF94FF43040009002208DF80500012082
:101AD0008DF8040000208DF8060001208DF8070025
:101AE00069461448FFF75CFD4FF4804000900020E9
:101AF0008DF8040001208DF8070069460D48FFF7B6
:101B00004FFD4FF48070009000208DF804000120FC
:101B10008DF8070069460848FFF742FD01221103CE
:101B20000448FFF7B9FD012251030248FFF7B4FD55
:101B30001CBD000000040240000C024070B50646C7
:101B4000002400224FF480512D48FFF7A5FD1420FA
:101B5000FFF7C7FB002523E000224FF4005128487F
:101B6000FFF79AFD06F0800028B10122D103244836
:101B7000FFF792FD05E000224FF400412048FFF7F7
:101B80008BFD1420FFF7ADFB012251031C48FFF72A
:101B900083FD7006060E1420FFF7A3FB681CC5B278
:101BA000082DD9DB1420FFF79CFB00251EE0002246
:101BB0004FF400511248FFF76FFD1420FFF791FB1F
:101BC0006006040E012251030D48FFF765FD4FF436
:101BD00080410B48FFF74FFD10B144F0010400E0D5
:101BE00000BF1420FFF77DFB681CC5B2082DDEDBAB
:101BF000012211030248FFF74FFD204670BD00008F
:101C00000004024070B505460E4600224FF4805194
:101C10002F48FFF741FD1420FFF763FB002423E06A
:101C200000224FF400512A48FFF736FD05F08000EE
:101C300028B10122D1032648FFF72EFD05E000223E
:101C40004FF400412248FFF727FD1420FFF749FB1E
:101C5000012251031E48FFF71FFD6806050E1420E0
:101C6000FFF73FFB601CC4B2082CD9DB1420FFF740
:101C700038FB002423E000224FF400511448FFF702
:101C80000BFD06F0800028B10122D1031048FFF7B8
:101C900003FD05E000224FF400410D48FFF7FCFC76
:101CA0001420FFF71EFB012251030948FFF7F4FC43
:101CB0007006060E1420FFF714FB601CC4B2082C3B
:101CC000D9DB012211030248FFF7E6FC70BD0000DA
:101CD0000004024000BFFEE730B502460B464FF657
:101CE000FF70521C15E0012110E000F0010424B146
:101CF000400844F20424604000E0400814780C409E
:101D000014B144F2042460404C06210E0029ECD1A9
:101D1000521C1C00A3F10105EBB2E4D130BD7047A9
:101D200008B54FF4A06000F04BF825208DF80000B6
:101D300000208DF801008DF8020001208DF80300CD
:101D4000684600F001F808BD70B5002100230F229D
:101D5000C4781CB3174C246804F4E064C4F5E06450
:101D6000C4F30721C1F10404E3B20A4144789C4062
:101D7000E1B28478144021430C07210E0E4C057803
:101D80006155047804F01F050124AC4005786D11FD
:101D9000AD0005F1E025C5F8004109E0047804F044
:101DA0001F050124AC40054D0678761145F8264004
:101DB00070BD00000CED00E000E400E080E100E018
:101DC00002490143024A1160704700000000FA0511
:101DD0000CED00E07047000029B1064A126802438A
:101DE000044B1A6004E0034A12688243014B1A60F4
:101DF000704700003038024029B1064A1268024399
:101E0000044B1A6004E0034A12688243014B1A60D3
:101E1000704700004038024029B1064A1268024368
:101E2000044B1A6004E0034A12688243014B1A60B3
:101E3000704700004438024029B1064A1268024344
:101E4000044B1A6004E0034A12688243014B1A6093
:101E50007047000024380240F0B500210022002421
:101E6000022500260223324F3F6807F00C0121B102
:101E7000042905D0082937D105E02E4F076036E048
:101E80002D4F076033E02A4F3F1F3F68C7F380564E
:101E9000274F3F1F3F6807F03F036EB1264FB7FB48
:101EA000F3F7DFF88CC0ACF1040CDCF800C0CCF325
:101EB000881C07FB0CF40CE01E4FB7FBF3F7DFF8B0
:101EC00070C0ACF1040CDCF800C0CCF3881C07FB3C
:101ED0000CF4174F3F1F3F68C7F301477F1C7D007D
:101EE000B4FBF5F7076002E0124F076000BF00BFC8
:101EF0000F4F3F6807F0F0010909104F7A5C07683F
:101F0000D74047600A4F3F6807F4E051890A0B4FFA
:101F10007A5C4768D7408760054F3F6807F46041A7
:101F2000490B064F7A5C4768D740C760F0BD000098
:101F3000083802400024F40000127A00000000205B
:101F400010B54FF400510248FFF7A0FB10BD000090
:101F5000000C024000B587B001210220FFF73CFFD2
:101F600001218804FFF748FF00208DF81A000120A6
:101F70008DF81B0003208DF8190002208DF8180041
:101F80004002059005A92E48FFF70AFB02208DF8B4
:101F900018008002059005A92948FFF701FB0121DF
:101FA0001020FFF719FF01208DF8180000208DF890
:101FB0001A0001208DF81B0003208DF819004FF442
:101FC0000040059005A91F48FFF7EAFA4FF40041C9
:101FD0001C48FFF75BFB07220A211948FFF728FB83
:101FE00007220B211648FFF723FB4FF416500190F0
:101FF0000020ADF80800ADF80A00ADF80C00ADF80F
:1020000010000C20ADF80E0001A90F4800F0CAFC2A
:1020100000F058F8012240F224410B4800F09CFCEB
:1020200001224021084800F057FC0121064800F039
:1020300047FC4FF400410348FFF726FB07B000BD03
:1020400000040240001002400048004000B58FB07C
:1020500001214805FFF7C0FE1748FEF7A5FE00BFA7
:102060001548FEF74DFF0028FAD14FF000600090B0
:10207000002003900A2004904FF480700990000221
:102080000A900E4801900020059007900E900C4891
:1020900002904FF480600690002008900D900B9005
:1020A00001200C9069460448FEF738FF01210248E0
:1020B000FEF76EFE0FB000BD2860024004480040ED
:1020C0009401002008B54FF4E060FFF779FE272067
:1020D0008DF8000001208DF801008DF802008DF8C8
:1020E00003006846FFF730FE08BD704730B5002298
:1020F0008B071C0F0F2303FA04F20B4B8C1053F8C1
:1021000024309343084C8D1044F8253023468C101E
:1021100053F824308C07240F00FA04F42343024CB4
:102120008D1044F8253030BD083801400CB5002032
:10213000019000903448006840F4803032490860D3
:1021400000BF3148006800F4003000900198401C46
:102150000190009818B90198B0F5A04FF1D12A4824
:10216000006800F4003010B10120009001E0002070
:1021700000900098012846D123484030006840F084
:1021800080502149403108602048006840F44040B8
:102190001E4908601C48083000681B490831086067
:1021A0000846006840F4004008600846006840F4B3
:1021B000A05008601648091F0860081F006840F01A
:1021C0008070091F086000BF0F48006800F00070B1
:1021D0000028F9D040F205700E4908600A4808301E
:1021E000006820F0030008490831086008460068CC
:1021F00040F00200086000BF03480830006800F0AB
:102200000C000828F8D10CBD0038024000700040D6
:1022100008544007003C024010B500F0BDFA10BD64
:1022200010B501F029FEFFF733FBFEF764FA00F06A
:102230004BF8FEF7FFFC01F0E9FBFFF73FFAFFF771
:1022400067F9FFF739FCFFF759FB002003490870D5
:102250005A2140F2CF7000F085F910BD57000020E0
:1022600010B51548006840F4700013490860134821
:10227000006840F001001149086000200F49083152
:1022800008600E4800680E4908400C4908600D4877
:10229000091D0860081F006820F48020091F0860DD
:1022A000002006490C310860FFF740FF4FF0006046
:1022B00001498039086010BD88ED00E00038024017
:1022C000FFFFF6FE103000241FB501210220FFF7AA
:1022D00093FD1D208DF8000001208DF803008DF87E
:1022E000010003208DF80200632002905320ADF816
:1022F00004000020ADF80600ADF80C0001A90A4862
:1023000000F008FA4FF4A060FFF75AFD6846FFF7A7
:102310001BFD01221146044800F0A8F901210248E2
:1023200000F087F91FBD00000004004010B5012136
:10233000704800F08AF900287ED06F480068401C81
:102340006D4908600846006801280FDB01206B49D1
:10235000086000206849086069480078022805D1B3
:1023600068480068022801DB00F01AFF6648006830
:10237000401C6549086008460068052805DB012007
:102380006249086000206049086061480068401C9C
:102390005F490860084600680A2805DB01205D499E
:1023A000086000205A4908605B480068401C5A4990
:1023B000086008460068B0F5FA7F4BDB01205749FA
:1023C000086000205449086055480068032841D13E
:1023D000544800685449554A128841F8220008467A
:1023E0005249098850F82100514909680844504968
:1023F000086000204B4908604E4800684E494B4A2F
:10240000128841F8220008464849098850F82100FE
:102410004A4909680844494908600020454908605C
:1024200042480088401C414908800846008814281A
:1024300010DB3F48006800E05BE0414908603F482E
:102440000068404908600020384908803849086021
:102450003A4908603C480068401C3B49086008460F
:102460000068B0F57A7F05DB01203849086000205C
:102470003549086036480068401C35490860084600
:10248000006841F28831884205DB0120314908604B
:1024900000202F49086030480068401C2E49086021
:1024A0000846006842F2107188421EDB144800782A
:1024B000022805D113480068401C124908600EE04C
:1024C0000F48007803280AD100200E4908604FF415
:1024D00000612248FFF7D8F802200949087001205E
:1024E0001F49086000201C4908600121014800F0D4
:1024F0009DF810BD000400401400002010000020D2
:1025000068000020480000201C0000201800002067
:1025100024000020200000202C00002028000020A3
:102520009800002014010020CC0300200E010020A0
:1025300018010020440100201C0400204801002054
:10254000100100203C010020340000203000002059
:102550003C0000203800002044000020001402400D
:102560004000002030B58BB005460C460121042008
:10257000FFF742FC01210820FFF72EFC4FF400403A
:10258000099002208DF8280000208DF82A000220F2
:102590008DF8290001208DF82B0009A91B48FEF7B2
:1025A000FFFF4FF400411948FFF76EF802220F2198
:1025B0001648FFF73DF8079540F24730ADF8180090
:1025C0000020ADF82000ADF81A0006A9104800F070
:1025D000A1F87020ADF804000120ADF8060002203B
:1025E000ADF81000039401A9094800F049F808214A
:1025F000074800F081F80121054800F00BF801219F
:10260000034800F016F80BB030BD0000000C02408B
:102610000008004021B1028842F08002028004E0FC
:1026200002884FF67F731A4002807047CA430282C5
:10263000704721B1028842F00102028004E0028862
:102640004FF6FE731A400280704730B502460020F4
:1026500000230024158A05EA0103958905EA01048F
:1026600013B10CB1012000E0002030BD1AB1838904
:102670000B43838102E083898B4383817047000091
:1026800070B5002200230024058C4EF6FF763540FD
:102690000584038C8488828B48F6FF752A404FF6A8
:1026A000FF452A400D884FF6FF7606EA05252A43A6
:1026B0004DF6FF752B408D8906EA05352B434D8875
:1026C00006EA05352B430A4DA84202D0094DA8421F
:1026D00008D14BF6FF752C400D8A4FF6FF7606EABF
:1026E00085152C43848082838D680564038470BDC6
:1026F00000000140000401400A460021818B4FF296
:10270000FF7319404FF6FF7303EA022319438183D5
:102710007047000000220288184B98420ED0184BD8
:1027200098420BD0B0F1804F08D0164B984205D09C
:10273000154B984202D0154B984204D14FF68F7337
:102740001A404B881A43124B984207D0114B9842BB
:1027500004D04FF6FF431A400B891A4302804B689E
:10276000C3620B880385054B984202D0044B984204
:1027700001D18B7A038601238382704700000140D8
:10278000000401400004004000080040000C00402C
:1027900000100040001400400448006820B10348C5
:1027A0000068401E0149086070470000500000208A
:1027B00010B504462146024800F063F910BD000040
:1027C0000010014000B587B001210846FFF704FB67
:1027D00001211020FFF720FB00208DF81A000120B6
:1027E0008DF81B0003208DF8190002208DF81800C9
:1027F0000002059005A91B48FEF7D2FE02208DF8C5
:1028000018004002059005A91648FEF7C9FE0722E8
:102810000A211448FEF70CFF072209211148FEF790
:1028200007FF4FF4E13001900020ADF80800ADF84B
:102830000A00ADF80C00ADF810000C20ADF80E0049
:1028400001A9094800F0AEF8FFF76AFA012240F248
:102850002551054800F080F80121034800F030F8C8
:1028600007B000BD000002400010014010B540F26A
:102870002551074800F046F840B10024044800F014
:10288000FBF8C4B2204601F0ADF800BF10BD000057
:102890000010014010B51021074800F026F801286B
:1028A00009D1FEF769FB054800F0A0FB024800884B
:1028B0000148001D008810BD004800409401002020
:1028C00021B1828942F40052828104E082894DF66E
:1028D000FF731A40828170471AB1838A0B43838247
:1028E00002E0838A8B438382704702460020B1F561
:1028F000007F00D100BF13880B400BB1012000E026
:102900000020704770B502460024002300250020F7
:1029100040F66A16B14200D100BFC1F3421501F082
:102920001F03012606FA03F3012D02D196893340D5
:1029300006E0022D02D1168A334001E0968A334028
:102940000C12012606FA04F41688344013B10CB1B7
:10295000012000E0002070BDF0B5034600240026F1
:102960000025002040F66A17B94200D100BF184682
:10297000C1F3421401F01F06012707FA06F5012CE6
:1029800001D10C3004E0022C01D1103000E01430F1
:102990001AB107682F43076002E00768AF4307607A
:1029A000F0BD00002DE9FF4705460E460024A14674
:1029B00000BFA046B08900B100BF2C8A24F4405467
:1029C000F08804432C82AC8941F20C608443B088C7
:1029D00031890843718908430443AC81AC8A24F4EB
:1029E0004074B0890443AC826846FFF735FA20484A
:1029F000854202D01F48854202D1DDF80C9001E0EB
:102A0000DDF80890A88900F4004040B109EBC90046
:102A100000EB091031684900B0FBF1F707E009EB62
:102A2000C90000EB091031688900B0FBF1F76420A0
:102A3000B7FBF0F004012009642101FB1078A8899C
:102A400000F4004040B1322000EBC800B0FBF1F0D0
:102A500000F00700044308E0322000EB0810642176
:102A6000B0FBF1F000F00F0004432C81BDE8FF87BC
:102A7000001001400014014001468888C0F308009E
:102A80007047C1F3080282807047000070B50546A8
:102A90000C464FF400411048FEF7F8FD0DE000BF72
:102AA0000E48008800F040000028F9D028780B4933
:102AB000091D08806D1C601EC4B2002CEFDC00BF35
:102AC0000648008800F040000028F9D04FF400418B
:102AD0000148FEF7D9FD70BD0010024000480040DB
:102AE0000021002200BF05E0002200E0521C7D2AE8
:102AF000FCD3491C8142F7D3704700BFFEE700B505
:102B00002DED048BB0EE409AF0EE609A83B051EC5C
:102B1000190BFDF760FD41EC180B18EE100A18EECA
:102B2000901A8DED008B002818BF0120084320F07B
:102B30000040C0F17F6000F1E040C00F14D019EEFA
:102B4000101A19EE900A8DED009B002918BF012183
:102B5000084320F00040C0F17F6000F1E040C00F6A
:102B600004BF012000F018F8B0EE480A03B0F0EE00
:102B7000680ABDEC048B00BD02E008C8121F08C142
:102B8000002AFAD170477047002001E001C1121FEE
:102B9000002AFBD17047000001490860704700001F
:102BA0009001002030B50B464049096889B90021E1
:102BB00000220BE03E4C34F81140240A84543C4C73
:102BC00014F81150541C0555491C921C1629F1DBB0
:102BD0001BE0002200210FE0364CA45C2CB90B2432
:102BE0004454B8254C1C055504E001244454F425F4
:102BF0004C1C0555521C891C142AEDDB282102E0CF
:102C000000224254491C2C29FADBF5EEC00AF1EEF1
:102C100010FA17DB002100F82C1F9FED271A20EE79
:102C2000811ABCEEC11A11EE101A090A41709FED0B
:102C3000221A20EE811ABCEEC11A11EE101A817010
:102C40002C381AE0012100F82C1FB0EEE01AF0EE4B
:102C5000410A9FED191A20EE811ABCEEC11A11EE3D
:102C6000101A090A41709FED141A20EE811ABCEE69
:102C7000C11A11EE101A81702C389FED101A20EE37
:102C8000011ABCEEC11A11EE101A090A00F82F1F22
:102C90009FED0A1A20EE011ABCEEC11A11EE101AAD
:102CA0004170012181702F3830BD0000500100209B
:102CB000B4020020B80300200000C84200007A449B
:102CC00000200DE00D4931F81010090A0C4B03F8F3
:102CD00010100A4911F810204100491C5A54401C98
:102CE0001428EFDB002006E006490A5C044B00F1E3
:102CF00028015A54401C1428F6DB70476C0400204D
:102D0000D00100209404002010B54A480078002823
:102D100044D14949086049480068494931F81000E0
:102D200040F2A32188420BDB4648007840B90120DD
:102D30004449087044480068401C434908600EE05C
:102D40003E4800683E4931F81000B0F5297F06DAA8
:102D50003C480078012802D100203A4908703B48DD
:102D60000068012864D100203849086038480068AC
:102D70005A2805DD36480068401E3549086005E0E0
:102D800001203449086000202F490860304800883D
:102D900081B240F2CF70FFF7E5FB49E027480068B9
:102DA000274931F8100040F2A32188420BDB254867
:102DB000007840B901202349087023480068401C6E
:102DC000214908600EE01D4800681D4931F81000D7
:102DD000B0F5297F06DA1B480078012802D10020CF
:102DE0001849087019480068012821D100201749A6
:102DF000086011480068142808D20F480068401C79
:102E00000D49086001211448FEF742FC1048006893
:102E100012490968884204D20D480068401C0C49D8
:102E200008600B48008881B240F2CF70FFF79AFB30
:102E300010BD00008200002024010020A800002016
:102E400084020020400100204401002038000020BE
:102E50003801002098000020001802409C0000204B
:102E60005B480068322817DA00200DE0594951F814
:102E70002010594A52F82020584B33F812201144A0
:102E8000544A42F82010401C1628EFDB50480068D6
:102E9000401C4F49086099E05148006814282CDA1A
:102EA0004C484F49096850F821003221B0FBF1F03D
:102EB0004C494B4A126841F8220000204549484AD3
:102EC000126841F822004749454A126831F8221039
:102ED00089B242F2107201FB02F0C11700EB1151EE
:102EE000C1F30F31404A3E4B1B6822F813103C4897
:102EF0000068401C3A49086068E0394800681428B6
:102F000031D134483649096850F821003221B0FBEC
:102F1000F1F13448324A126840F8221000202D495D
:102F20002F4A126841F822002E492D4A126831F8C2
:102F3000221089B240F6B83201FB02F0C11700EB53
:102F40001151091301EB81014FF6FF7202EA4102B0
:102F50002549234B1B6821F8132021480068401C99
:102F60001F49086032E01E48006815282ED1194814
:102F70001B49096850F821003221B0FBF1F11948D2
:102F8000174A126840F8221000201249144A1268A9
:102F900041F822001349124A126831F8221089B20E
:102FA00040F6B83201FB02F0C11700EB11510913D2
:102FB0004FF6FF7202EA81010B4A094B1B6822F8A7
:102FC000131000200649086001490860704700009E
:102FD0000001002060030020A800002084020020DF
:102FE0000401002008030020B40200200121204A2F
:102FF00011704178022918D18178032915D181797E
:1030000009021C4A1160C17912681143194A116002
:10301000114691ED000AB8EE400ADFED170A80EE86
:10302000201A164981ED001A1AE04178A02917D11B
:103030008178202914D1417909020E4A11608179E1
:10304000126811430B4A1160114691ED000AB8EE67
:10305000400ADFED090A80EE201A084981ED001AC6
:10306000064991ED000A064981ED000A704700000B
:10307000840100208801002000007A448C01002097
:103080005801002010B510214048FEF7F4FA4049DD
:10309000087020213D48FEF7EEFA3D494870402176
:1030A0003A48FEF7E8FA3A49887080213748FEF737
:1030B000E2FA3749C8704FF400713648FEF7DBFA80
:1030C000334908714FF480613248FEF7D4FA304931
:1030D00048714FF400612F48FEF7CDFA2C498871F2
:1030E0004FF480512B48FEF7C6FA2949C8714FF4B6
:1030F00000512848FEF7BFFA254908724FF4804175
:103100002448FEF7B8FA224948724FF4004121489A
:10311000FEF7B1FA1E49887208211F48FEF7ABFA84
:103120001B49C87210211C48FEF7A5FA18490873FC
:1031300020211948FEF79FFA154948734021164887
:10314000FEF799FA1249887380211348FEF793FA23
:103150000F49C8734FF480710F48FEF78CFA0C4981
:1031600008744FF400710C48FEF785FA084948745A
:1031700001210A48FEF77FFA0549887402210748B1
:10318000FEF779FA0249C87410BD0000000C024035
:10319000B803002000180240000402400010024062
:1031A00010B54FF400611A48FEF770FA194800682C
:1031B00001282CD100201749086017480068401CDE
:1031C000154908600846006842F2107188421ADD0D
:1031D00012480068401C1149086000200E49086030
:1031E0000F4908600F4908600C480068142806DB86
:1031F00004200D49087000200849086007E00320FA
:103200000949087003E00548006800F077FD10BD2B
:103210000014024010000020700100207401002002
:10322000680100206C0100206800002010B5FEF746
:10323000ADF900F085FA00F053FA154890ED000A58
:10324000DFED140AB4EEE00AF1EE10FA1ED800F039
:1032500091FA114800684FF6FF71884204D20E4877
:103260000068401C0C4908600B48006842F210716D
:10327000884204D201210948FEF708FA06E001213C
:103280000648FEF701FA00200549087010BD00004D
:10329000600100200AD7233C2401002000180240CE
:1032A0008100002010B5FEF74BFE00F049FA00F057
:1032B00017FA4FF480511248FEF7DDF9F0B900F02B
:1032C00059FA104800684FF6FF71884204D20D4841
:1032D0000068401C0B4908600A48006842F21071FF
:1032E000884204D201210848FEF7D0F906E0012106
:1032F0000548FEF7C9F900200449087010BD000018
:10330000001002402401002000180240810000202B
:1033100010B506480068012806D10020034908605E
:1033200002210348FEF7B4F910BD00004000002060
:1033300000180240FEF774FF03E000F003F8FFF707
:10334000E7FFFAE710B518480068012804D0022802
:1033500005D0032809D105E000F02EF806E000F0C2
:10336000EFF803E000F09EF800E000BF00BFFDF7BB
:1033700099FE0E4800680A3800EE100AB8EE400ABE
:10338000DFED0B0A80EE201AB1EE040A31EE400A9E
:10339000F0EE000A80EE201A064880ED001A90ED4B
:1033A000000AFDF713FC10BD9800002090000020DB
:1033B0000000C8426401002010B52E480068401C7F
:1033C0002C49086008460068322807DD2A48FDF7C6
:1033D000D3FBFFF745FD0020264908602748006819
:1033E000022802D1FDF7F2FD01E000F0B9FB24480C
:1033F000007810B100202249087022480068012896
:103400000BD100201F490860FEF77EFA1E4880EDB0
:10341000000A08211D48FFF739FBFFF733FE1C485F
:1034200090ED000AB5EEC00AF1EE10FA0BD1194882
:1034300090ED000A1648D0ED000A30EE600A1648FA
:1034400080ED000A0AE0124890ED000A1148D0ED24
:10345000000A30EE600A104880ED000A0A48D0EDFC
:10346000000A0D4890ED000A0C490D48FFF79AFB41
:1034700010BD00008001002000200140200100203C
:103480005700002030000020540100207801002067
:103490005C0100205801002060010020B4020020DF
:1034A0009E01002010B51E480068401C1C490860A1
:1034B000084600680A2805DD1A48FDF75DFB002074
:1034C00017490860FFF720FC17480068012826D13B
:1034D00000201549086015480088000A1449087042
:1034E00012480078487013480088000A8870114814
:1034F0000078C8700B4604220F4801884FF2030081
:1035000000F0C4FA0B480068B0F57A7F07DD074881
:103510000068B0F57A7F02DD00200849087010BD10
:103520008001002000200140300000201001002018
:10353000590000203C01002066000020820000208D
:1035400010B55348FDF718FB5248007801287DD18B
:1035500051480068012806D100204F490860082121
:103560004E48FFF793FA4E4890ED000AB5EEC00AB8
:10357000F1EE10FA0BD14B4890ED000A4848D0ED1F
:10358000000A30EE600A484880ED000A0AE044482C
:1035900090ED000A4348D0ED000A30EE600A424840
:1035A00080ED000A404890ED000A4048D0ED000A46
:1035B000B4EEE00AF1EE10FA02DDFDF7E7FF01E0FC
:1035C000FEF7BEFC00F0BCF800F0A2F8374890ED22
:1035D000000ADFED370A30EE200A3348D0ED000A4A
:1035E000B4EEE00AF1EE10FA3DDD304890ED000A4D
:1035F000DFED2F0A30EE600A2B48D0ED000AB4EE62
:10360000E00AF1EE10FA2ED200F0B4F800201BE030
:103610000021284A22F81010274A22F81010274AC1
:103620001154274A52F82020264B33F8122042F238
:10363000107302FB03F1CA1701EB1252C2F30F32EF
:10364000214B23F81020401C142800E00BE0DFDBA6
:103650004FF400611D48FEF717F800201C49086070
:1036600002200C4908700B48007804280FD1002074
:1036700008490870FFF724FB164B3C2216480188C6
:103680004FF2020000F002FA01201449086010BD58
:103690000020014068000020300000207801002058
:1036A0005C0100205801002060010020A4000020DF
:1036B000CDCC4C3DA80400206C04002094040020D4
:1036C000A800002084020020E00200200014024034
:1036D00074010020D0010020660000209800002026
:1036E00010B50848006860B10020064908604FF432
:1036F00080510548FDF7CCFF04480068401C034991
:10370000086010BD18000020000C02402C010020B1
:1037100010B50848006860B10020064908604FF401
:1037200080510548FDF7B4FF04480068401C034978
:10373000086010BD20000020000C02402C01002079
:103740001CB501210820FEF747FB4FF48050009084
:1037500001208DF8040000208DF806008DF8070088
:103760008DF8050069460248FDF71AFF1CBD0000F0
:10377000000C02401CB501210820FEF72DFB4FF480
:103780008050009000208DF804008DF807008DF81F
:10379000050069460148FDF703FF1CBD000C02400F
:1037A00010B57548006800B910BD74480078072846
:1037B0007DD2DFE800F0DC04152D8288B600002001
:1037C0006F4908606F4908606F4890ED000A6F48C4
:1037D00080ED000A69480078401C68490870C7E01D
:1037E000FFF7AEFFFFF794FF6348006800EB80002F
:1037F00063490968B1EB001F09D3002060490860E4
:10380000FFF7B8FF5D480078401C5C490870AFE0E6
:103810005F48006838B100205D490860584800687A
:10382000401C57490860564800685A490968884250
:1038300042D3002052490860534890ED000A564890
:1038400080ED000A90ED000A5048D0ED000A30EEFD
:10385000600AB0EEC00ADFED510A60EE200A464869
:10386000006800EB80000121C1EB400000EE100A6F
:10387000B8EE400AF4EEC00AF1EE10FA03D20520C9
:103880003E49087018E03D480078401C3B490870EC
:103890004348D0ED000A434890ED000A42494348AE
:1038A000FFF780F9414B32224148018800E05EE099
:1038B0004FF2010000F0EAF85AE000202F490870AA
:1038C0003C49087054E0FFF73BFFFFF721FF324807
:1038D00090ED000A2D48D0ED000A30EE600AF0EEBF
:1038E000C00A254890ED000AB8EE400A9FED321A52
:1038F00000EEC10ADFED310A60EE200A204890EDAB
:10390000000AB8EE400AF4EEC00AF1EE10FA07D849
:1039100000201B490860FFF72DFF0620174908709B
:1039200026E01B48006838B1002019490860144897
:103930000068401C12490860114800681549096870
:10394000884213D300200E4908600F4890ED000A0A
:10395000114880ED000A042008490870134B3222F8
:10396000134801884FF2010000F090F800E000BF1A
:1039700000BF00BF18E700008800002028010020D9
:103980002C0100201C0100205801002030010020E3
:10399000200000208C0000203401002000007A4428
:1039A0005401002060010020B40200209E0100208C
:1039B00066000020810000200000C8420000A042F4
:1039C00000B50020044908700449087004490870D3
:1039D000FDF75EFF00BD00005F00002060000020DA
:1039E0006100002010B50446074800783C2806DA3C
:1039F0000A2000F071F92046FDF780FC03E0FFF794
:103A0000DFFFFDF745FF10BD5E0000201CB5002064
:103A10008DF804004FF40060009002208DF805003E
:103A200000208DF8070001210820FEF7D5F9F020CD
:103A3000009069461148FDF7B3FD01214020FEF7D3
:103A4000CBF94FF47E40009069460D48FDF7A8FD84
:103A500001210220FEF7C0F94FF47E700090694604
:103A60000848FDF79DFD01211020FEF7B5F9032060
:103A7000009069460448FDF793FD1CBD000C024010
:103A80000018024000040240001002402DE9F043FB
:103A90008FB006460F46144698464FF000090025A1
:103AA00005208DF8000004F10B00C11700EB116137
:103AB000090A8DF80110C11700EB11610912A0EB82
:103AC0000121C9B28DF80210380A8DF80300F8B24E
:103AD0008DF8040021480088000A8DF805001F4871
:103AE00000788DF80600300A8DF80700F0B28DF8E6
:103AF000080000BF07E018F8051005F109000DF8EF
:103B00000010681CC5B2A542F5DB04F10800C1B283
:103B10006846FEF7E1F8814609F0FF0104F109006B
:103B20000DF80010C9F30721401C0DF800101B21EF
:103B3000401C0DF80010002508E01DF80500FEF7F8
:103B400037FE3220FEF7CCFF681CC5B204F10C0032
:103B50008542F2DB0FB0BDE8F08300006400002076
:103B600010B52DED068B9FED4B0AB0EE408A4A480A
:103B7000006858BBFDF70AFDFFF7E2FDFFF7C8FD3F
:103B80004FF400614548FDF776FD00281DD14449FA
:103B900008704448006838B1002042490860424833
:103BA0000068401C404908603F480068B0F5FA7F53
:103BB0006ED300203C4908603C4890ED000A3C4828
:103BC00080ED000A01203449086061E03248006855
:103BD00001285AD1374890ED000AF3EE0E0AB4EEF0
:103BE000E00AF1EE10FA14DD33490978491C480067
:103BF000FCF7FCFB41EC1A0B9FED300B53EC102B48
:103C0000FCF7DEFA41EC190BFCF714FC08EE100A85
:103C100009E029480078401C400000EE100AB8EE88
:103C2000C00AB0EE408A274890ED000AB4EEC80AF8
:103C3000F1EE10FA22DB2448006842F2107188424B
:103C400009D221480068401C1F49086001211F4813
:103C5000FDF71CFD1CE001211C48FDF715FD0020AF
:103C60000F49087002200C490860194B322219488C
:103C700001884FF20400FFF709FF09E0FEF760F941
:103C8000FFF75EFDFFF744FD02E0BDEC068B10BDC3
:103C900000BFFAE7000000002001002000100240F1
:103CA00081000020200000202C010020580100206D
:103CB0005C010020540100208000002033333333A6
:103CC0003333C33F6001002024010020001802406C
:103CD0009E0100206600002000B970470121044ABF
:103CE00011700021034A1170034A107000BFF4E7FD
:103CF0005F000020600000206100002030B5564BBE
:103D000033F81030C3EB0313C3EBC303642493FBFA
:103D1000F4F4524B53F82030514D35F8133042F241
:103D2000107503FB05F2D31702EB13531B139C42D0
:103D300027DB494B33F81030C3EB431404EB8313F8
:103D4000642493FBF4F4454B53F82030444D35F88C
:103D5000133042F2107503FB05F1CB1701EB13533F
:103D60001B139C420DDC3F4B33F810304BB93E4BDC
:103D70001B68032B05DD3C4909883A4A22F81010DC
:103D80000EE039490968491C374A11601146096833
:103D900047F23052914203DD4FF6FF71324A116013
:103DA0002D4A32F81020C2EB0212C2EBC202642389
:103DB00092FBF3F3294A52F82020294C34F81220C0
:103DC00042F2107402FB04F1CA1701EB12521213F3
:103DD000934207DA254A32F810201AB90121234A02
:103DE00022F81010214931F81010012932D11A4A55
:103DF00032F81020C2EB0212C2EBC202642392FB23
:103E0000F3F3164A52F82020154C34F8122042F2EF
:103E1000107402FB04F1CA1701EB12521213934201
:103E20000BDB134A125C42B90221104A22F810102F
:103E3000104909780E4A11540CE00E490968FF290F
:103E400003DDFF210B4A116004E00A490968491C9F
:103E5000084A116030BD0000E0020020A8000020E8
:103E6000840200206C04002068010020A8040020C7
:103E7000940400206C01002010B5FDF751FFFEF7FF
:103E8000A1FCFEF71FF9FEF765F8FEF7DFF810BD9D
:103E9000B03E00080000002094010000BC060008AD
:103EA000043F0008940100203C070000882B000814
:103EB000510D550102030401020304060708090419
:103EC0002AA100B17334030210014213420D4204CF
:103ED000420142094206820342154212420F420C3D
:103EE000420E420B4208420542024217421442115E
:103EF000420702240A02180202405A430203041530
:043F000002C43800BF
:040000050800018965
:00000001FF
